:100000000C946D000C948A000C948A000C948A0065
:100010000C948A000C948A000C948A000C948A0038
:100020000C948A000C948A000C948A000C948A0028
:100030000C948A000C948A000C948A000C948A0018
:100040000C948A000C948A000C948A000C948A0008
:100050000C948A000F00070107040303030607023C
:1000600006030103020100202122111111110003D6
:1000700001010111111111111111000312020000EF
:1000800012121111111100031212000200101111AD
:10009000111102011010212201010111111102039D
:1000A00010100112020010111111020310000102C0
:1000B000222010111111000312120001011111115F
:1000C000111100031212000002222020111102015E
:1000D0001020220201001011111111241FBECFE5C2
:1000E000D8E0DEBFCDBF10E0A0E6B0E0ECE7F4E181
:1000F00002C005900D92A237B107D9F713E0A2E72D
:10010000B0E001C01D92AE30B107E1F70E94FB00E4
:100110000C943D0A0C9400008FE085BD14BC8EE465
:1001200083BD089508B607FEFDCF80E888BF089517
:100130008BB38F638BBB8AB3807C8ABB10927200B7
:100140001092730010927400089529B320952F73B4
:1001500080917300281741F02093730081E0809311
:10016000740080E090E0089580917400882369F025
:10017000815080937400882341F4809172008095AF
:100180008223209372009927089580E090E00895DB
:100190000E94A500992782FD16C083FD09C084FD39
:1001A00017C080917200992785FF0BC022E015C00F
:1001B00060E081E00E94860780917200992785FDAA
:1001C000F5CF20E00AC060E08FEF0E948607E9CFFC
:1001D00061E080E00E948607E4CF96958795817064
:1001E000282B20930D030E9479078091AE00805F39
:1001F0008093B40008951F930E948C000E944E01CA
:100200000E9483050E94980010E808B607FEFDCF03
:1002100018BF0E94C800F9CF08B601FEFDCF82E0EA
:1002200088BF089582BB65BB0895982F22E008B669
:1002300001FEFDCF28BF82B3890F82BB6150B9F7A1
:100240000895982F22E008B601FEFDCF28BF85B3A0
:10025000890F85BB6150B9F70895EF92FF920F9314
:100260001F93F82EE62E142F022F0E9412011F1941
:10027000612F81E00E9415010E19602F81E00E941C
:100280002101612F8FEF0E941501602F8FEF0E94D7
:1002900021011F910F91FF90EF90089589E083BF96
:1002A00012BE84E18CBF60E080E00E9412018FEFFB
:1002B00081BB84BB0895982F22E008B601FEFDCFD4
:1002C00028BF82B3890F82BB85B3860F85BB41509F
:1002D000A1F7089508951F93CF93DF93DC01FB01ED
:1002E000442309F46EC061E040E050E0EC0123815A
:1002F00082818623D9F032E081818623D9F074E0AF
:1003000080818623D9F098E080E0262309F081E0FF
:10031000372B932B892B89934F5F5F4F44305105C7
:1003200079F0660F23818281862329F730E081816D
:10033000862329F770E08081862329F790E0E4CFB7
:100340008481ED018C8385818D83EC911E2F6A81E0
:10035000462F55277B81872F9927482B592BF981C9
:100360008F2F99272E2F3327822B932B482B592BF6
:1003700040FD16C0E12FE695F6956695ED016A837E
:1003800076957B831E2F8E2F99272F2F3327822B35
:10039000932B272F262B282B20FFECCFF983EC93D0
:1003A000EE2309F03CC0FD018181982F862F672F35
:1003B000ED017A8370E01B829923B9F389839C93C2
:1003C0002EC068E040E050E0EC012081818186236E
:1003D000E1F032E082818623E1F074E083818623BC
:1003E000E1F098E080E0262309F081E0372B932BA1
:1003F000892B89934F5F5F4F4430510509F4A0CF9B
:10040000669520818181862321F730E082818623D1
:1004100021F770E08381862321F790E0E3CFDF911D
:10042000CF911F910895FC0140815181942F952B0C
:1004300022813381822F832B982B99F0442371F4EE
:100440008581952F492F922F232F328330E01382FD
:100450008F5F85834423B1F39183408381E090E0F3
:10046000089580E090E008951F93E3E8F0E081E0D4
:1004700098E08193919320E0EB3AF207D1F7109145
:10048000B100112379F150E0852F9927FC01EE0F7F
:10049000FF1FE80FF91FEE0FFF1FEB54FF4F848182
:1004A0008F5F682F772767FD70958581A82FBB2701
:1004B000AA0FBB1FAD57BF4F40E021913327062E37
:1004C00002C0220F331F0A94E2F78D919C9111977D
:1004D000822B932B8D939D934F5F443071F75F5F19
:1004E000151791F61F910895FC0184818F5F682F85
:1004F000772767FD70958581A82FBB27AA0FBB1FA3
:10050000AD57BF4FAF014C5F5F4F21913327062E90
:1005100002C0220F331F0A94E2F78D919C9111972C
:10052000822793278D939D93E417F50771F708951C
:10053000CF93DF93FC0184818F5FC82FDD27C7FD38
:10054000D0958581A82FBB27AA0FBB1FAD57BF4FE2
:1005500040E050E0BF016C5F7F4F819199270C2EE6
:1005600002C0880F991F0A94E2F72D913D918223D2
:100570009323482B592BE617F70779F780E090E093
:10058000452B11F481E090E0DF91CF910895CF9257
:10059000DF92EF92FF920F931F93CF93DF933091EF
:1005A000B1003323E1F020E040E0822F9927FC01E5
:1005B000EE0FFF1FE80FF91FEE0FFF1FEB54FF4F69
:1005C0009481892F807F19F09051948341E02F5FAF
:1005D000231759F7442319F0842F99274AC0EE2492
:1005E000FF24E3E8F0E008C00894E11CF11C329617
:1005F00024E1E216F104D9F1808191818150984083
:1006000099F73323A1F1DD2420E076E0C72E03C063
:10061000D394D31648F58D2D9927EC01CC0FDD1F0F
:10062000C80FD91FCC0FDD1FCB54DF4F8D81992709
:1006300087FD9095E816F9065CF7DC9C8001112493
:100640000B541F4FC8010E9474028D8181508D830D
:10065000C8010E9474028C81806A8C8321E03091F1
:10066000B100D394D316B8F2822F992702C080E04C
:1006700090E0DF91CF911F910F91FF90EF90DF906D
:10068000CF900895EF92FF920F931F93CF93DF9334
:100690003091B100332309F456C020E0EE24822FBC
:1006A0009927FC01EE0FFF1FE80FF91FEE0FFF1F48
:1006B000EB54FF4F9481892F807F21F090519483D8
:1006C00041E0E42E2F5F231751F7EE20C9F5FF24F8
:1006D0000DC0C8010E9474028C81806A8C8311E075
:1006E000E12E3091B100F394F31650F58F2D992738
:1006F000EC01CC0FDD1FC80FD91FCC0FDD1FCB5471
:10070000DF4F8D8118167CF786E0F89E800111245A
:100710000B541F4FC8010E9474028D8181508D833C
:10072000C8010E9498028823A1F68D818F5F8D8376
:10073000C8010E9474023091B100F394F316B0F234
:100740008E2D992702C080E090E0DF91CF911F911C
:100750000F91FF90EF90089580E090E0E3E8F0E0E3
:1007600006C0C901019632968431910539F09C0189
:10077000808191818F5F9F40A1F702C02FEF30E011
:10078000C9010895643098F4443088F4A42FBB273D
:10079000A7FDB095A80FB91FE62FFF27E7FDF0953D
:1007A000E05AFF4F8C91908189239927089580E02A
:1007B00090E008956DEC81E30E94120162E382E013
:1007C0000E94150164E68EEF0E94210162E38EEF24
:1007D0000E94150164E682E00E9421010895AF9213
:1007E000BF92CF92DF92EF92FF920F931F93CF931E
:1007F000DF93EC01988180916000892309F08BC020
:1008000080916100892309F08EC080916200892364
:1008100009F083C080916300982309F081C0F4E05F
:10082000AF2E6F3F09F46EC08C812D815AE0259F59
:1008300090011124482F42954F70640F695F620F39
:100840008F708A0D859FC00111248C5C0E9412015B
:10085000DA2C71E0F72EEE24BB24CF2C0D2D0E0DDB
:10086000043098F4AB2DAF19A43078F4BB27A7FD62
:10087000B095AC0FBD1FE02FFF27E7FDF095E05AC4
:10088000FF4F8C919081892349F51F2D1D0D143048
:10089000A0F40B2D0E0D043080F4A02FBB27A7FD74
:1008A000B095AC0FBD1FE12FFF27E7FDF095E05A93
:1008B000FF4F8C9190818923E9F446E06E2D8F2DB6
:1008C0000E945B01FE2CF194EC2C81E0F81629F6D5
:1008D000EE2019F6BB2009F0C0CF28C01F2D1195BE
:1008E00044E0612F8E2D0E945B01B10EFE2CE12EA3
:1008F000D02EEBCF4AE06E2D8F2D0E945B01D12EC2
:10090000B02EE3CF8AE0A89EC001112464EB865F7D
:100910000E9412019DCFAA2484CFA2E0AA2E81CFEB
:10092000E3E0AE2E7ECFB1E0AB2E7BCFDA1409F040
:1009300094CFDF91CF911F910F91FF90EF90DF90B7
:10094000CF90BF90AF900895BF92CF92DF92EF9279
:10095000FF920F931F93CF93DF9384E18CBF80911D
:10096000B100882379F000E016E0019FC001112456
:1009700060E08B549F4F0E94EF030F5F8091B100A6
:10098000081798F38091B20080FD68C081FF1BC0FA
:1009900082E38CBFC3E8D0E008E004C02296065F83
:1009A000003D79F08881998197FFF8CF202F2C5F47
:1009B00044E9602F85E30E942D012296065F003DE9
:1009C00089F784E18CBF6FEF85E790E00E94EF0329
:1009D0008091B20082FF4FC06091B300B62EB694F2
:1009E000B6940091AD00112766957727882777FD8B
:1009F0008095982F0E9489099B01AC0160E070E00E
:100A00008BE193E40E9429090E946C096B017C012F
:100A10006B2D7727882777FD8095982F0E9489096D
:100A20009B01AC0160E070E088EC92E40E9429092F
:100A30000E946C09DC01CB0198014B2D6C2D0E94AA
:100A400035088091B30081508093B300853099F4CC
:100A50008091B2008B7F8093B2000DC060918100C5
:100A600070918200672F77278BE790E00E94EF0359
:100A70008091B2008BCF2091AB003091AC0044E06C
:100A80006BE98AE00E9435082091AE003091AF00FA
:100A900044E067E88AE00E9435088AE08CBF0E9443
:100AA000DA03DF91CF911F910F91FF90EF90DF90CC
:100AB000CF90BF900895ABE7B0E0E5E7F0E086E0C7
:100AC00001900D928150E1F70E94190987708730DB
:100AD000D9F39927880F991FFC01EC5AFF4FE49135
:100AE000E09375008B5A9F4FFC01849180937600B0
:100AF000109277001092780084E08093790082E170
:100B000080937A0008951092B1001092B200109272
:100B1000AC001092AB001092AF001092AE0081E0DA
:100B20008093B00010920D0380E18093B4000E9486
:100B300034020E945B050895DB01FA0136E0019062
:100B40000D923150E1F7DC01FA0136E001900D928F
:100B50003150E1F740E050E0FB01E40FF11D10825D
:100B60004F5F5F4F2417C0F7243038F4FC01E20FC9
:100B7000F11D10822F5F2430C9F70895582F40913E
:100B8000B100282F3327842F992701972817390779
:100B90007CF486E0589FD0011124489FF001112475
:100BA000AB54BF4FE155FF4F01900D928150E1F7DB
:100BB00041504093B1000895AC012091B10024361A
:100BC00008F0089586E0289FF0011124EB54FF4FB0
:100BD000DA010D9001928150E1F72F5F2093B1006F
:100BE0000895AF92BF92CF92DF92EF92FF920F9350
:100BF0001F93CF93DF93CDB7DEB72C970FB6F89442
:100C0000DEBF0FBECDBFE82E3091B100332309F413
:100C10005BC0FF2467E0C62ED12CCC0EDD1E5E012A
:100C20000894A11CB11C04C0F394F31608F04CC046
:100C30008F2D9927FC01EE0FFF1FE80FF91FEE0F14
:100C4000FF1FEB54FF4F85812E2D281B243060F7AA
:100C500086E0F89E800111240B541F4FA801B501B6
:100C6000C6010E949C05C6010E941302882391F0D0
:100C7000F801D60186E00D9001928150E1F7C5019F
:100C80000E9413028823D1F43091B100F394F3163B
:100C900078F21AC0C5010E941302882341F0F801BE
:100CA000D50186E00D9001928150E1F7EDCF8F2DB7
:100CB0000E94BE05FA943091B100B6CFC5010E94E2
:100CC000DC053091B100B0CFEE2DFF27E7FDF095A8
:100CD000EE0FFF1FED57FF4F81E098E09183808377
:100CE0002C960FB6F894DEBF0FBECDBFDF91CF912B
:100CF0001F910F91FF90EF90DF90CF90BF90AF903A
:100D00000895FF920F931F938091B000813009F4F2
:100D1000B4C0823051F0833009F443C0843009F408
:100D2000C3C0853009F0E1C088C080910D0380FF09
:100D300092C020918100309182002C5F334030932B
:100D400082002093810037FFD0C02050364F30936F
:100D500082002093810090918000915090938000B8
:100D600097FD09C08BE790E00E949802882309F064
:100D7000BCC0909180008091B2008E7F8093B200C1
:100D80009F5F909380008BE790E00E94DC058BE7EB
:100D900090E00E9474021092AD0083E08093B00056
:100DA000A4C081E08093B000E5E0FE2E04E117C00E
:100DB000812F0E94F105E12FFF27EE0FFF1FED5756
:100DC000FF4F808191819068918380838091AD00F5
:100DD0008F5F8093AD00F092B0000093B3000E944B
:100DE000AC03182F8F3F21F78091B000813009F0BC
:100DF0007CC02091AD00222309F477C08091AB0024
:100E00009091AC00820F911D9093AC008093AB0049
:100E10008091AE009091AF0001969093AF008093C7
:100E2000AE00243008F461C08091B20084608093E9
:100E3000B20084E68093B30058C08091B300815023
:100E40008093B300882309F446C08091B200826089
:100E50008093B2004AC08091B4009927880F991FEF
:100E6000880F991F2091810030918200281B390B37
:100E7000309382002093810066CF0E945B0520E0C2
:100E80003AE030938200209381008BE790E00E944B
:100E900098028823A9F08091B20081608093B2000B
:100EA00082E08093B00021C080910D0381FF10C0CB
:100EB0000E944203882341F084E08093B00015C073
:100EC0008FEF8093B00011C083E08093B0000DC01D
:100ED0000E94C702EFCF0E94340284E08093B000EA
:100EE0008091B2008D7F8093B2001F910F91FF908F
:100EF00008950E94A4040E9481060895DC01FB016C
:100F000086E001900D928150E1F708950F931F93B1
:100F1000CF93DF93CDB7DEB726970FB6F894DEBF39
:100F20000FBECDBF182F062F882329F5002309F403
:100F30005DC040E06BE770E08E010F5F1F4FC8019E
:100F40000E946B01C8010E949802882329F58D81B7
:100F5000833008F44BC081508D83C8010E949802F1
:100F6000882319F1ABE7B0E0F80186E001900D921B
:100F70008150E1F73BC080917F00810F80937F001B
:100F80008BE790E00E949802882381F680917F0091
:100F9000811B80937F00CACFABE7B0E0F80186E009
:100FA00001900D928150E1F721C08D8181508D8398
:100FB000C8010E949802882389F48D8181508D8315
:100FC000C8010E949802882389F0ABE7B0E0F801DD
:100FD00086E001900D928150E1F708C0ABE7B0E0E8
:100FE000F80186E001900D928150E1F726960FB648
:100FF000F894DEBF0FBECDBFDF91CF911F910F914F
:101000000895FF920F931F93CF93DF93562FF42EE3
:1010100089010F5F1F4FF801649101501040F801E2
:101020009491649F602D1124650F499F902D112488
:10103000890F0E941201E8012296FE0184918131FC
:1010400071F0682F62956F7061508F704F2D8150D5
:101050000E945B012196FE018491813191F7DF911D
:10106000CF911F910F91FF900895AF92BF92CF92B1
:10107000DF92EF92FF920F931F93CF93DF93D82EBF
:10108000B62E142F790124E030E0ECE6F0E0C22E19
:1010900080819181E816F90638F42150304032976A
:1010A00021153105A1F7CC2483E0189FA02C112431
:1010B000EC2DFF27EE0FFF1FEC59FF4F0190F08141
:1010C000E02DEE16FF0608F441C0442755274E1BBD
:1010D0005F0B97012E1B3F0B00E00F5F240F351FA6
:1010E000CF01820F931F8E179F07B8F77C018CE00A
:1010F000089FE0011124CE59DF4F2196FE01649133
:101100002197FE018491169F602D11246B0D189F6D
:10111000802D11248D0D0E9412012296FE018491D2
:10112000813171F0682F62956F7061508F70412F1F
:1011300081500E945B012196FE018491813191F7DB
:10114000013011F0DA0C06C0D10E04C000E0C2E696
:10115000D0E0D3CFCA94FFEFCF1609F0A9CFDF912B
:10116000CF911F910F91FF90EF90DF90CF90BF90A4
:10117000AF900895AF92BF92CF92DF92EF92FF921D
:101180000F931F93CF93DF93EC01A880B980CA809F
:10119000DB80A114B104C104D10449F482E4E82E37
:1011A0008EECF82E8CE0082F8FE1182F2EC0C60190
:1011B000B5012DE133EF41E050E00E94000A27EA3B
:1011C00031E440E050E00E94E1097B018C01C6015E
:1011D000B5012DE133EF41E050E00E94000ACA0161
:1011E000B90124E13BE040E050E00E94E109E61A49
:1011F000F70A080B190B17FF08C08FEF9FEFAFEF2F
:10120000BFE7E80EF91E0A1F1B1FE882F9820A8356
:101210001B83C7019F77DF91CF911F910F91FF90A3
:10122000EF90DF90CF90BF90AF9008950E94BA08E2
:1012300008958EE690E00E94BA080895AA27BB2779
:1012400080936E0090936F00A0937000B093710034
:1012500008955058192E84D001D06AC0BA17620779
:10126000730784079507B1F188F40EF410940B2EE0
:10127000BA2FA02D062E622F202D072E732F302D72
:10128000082E842F402D092E952F502DFF275523F2
:10129000B9F0591B49F0573E98F046953795279578
:1012A000A795F0405395C9F776F0BA0F621F731FE8
:1012B000841F30F4879577956795B795F04093959F
:1012C00017FA0F2E0895BF1BBB27BA0B620B730BC7
:1012D000840BF6CFDEF670C097FB4ED09F3738F008
:1012E000FEE9F91B982F872F762F6B2F05C061C061
:1012F0009695879577956795F150D0F73EF4909540
:101300008095709561957F4F8F4F9F4F0895E8941A
:1013100003C097FB0EF4F3DFB62F672F782F892FCA
:101320009EE9002405C09A95BB0F661F771F881F92
:1013300011249923A1F08823B2F79F3F59F0BB0FE6
:1013400048F421F4002011F460FF04C06F5F7F4F68
:101350008F4F9F4F881F9795879597F9089529C0BC
:10136000052E092607FA440F551F5F3F79F0AA277B
:10137000A51708F051E04795880F991F9F3F31F05E
:10138000BB27B91708F091E0879508959F919F9129
:10139000112414C097FB880F991F9F3F31F0BB2782
:1013A000B91708F091E0879508959F919F911124B6
:1013B00005C0662777278827992708959FEF80EC37
:1013C0000895629FD001739FF001829FE00DF11D8F
:1013D000649FE00DF11D929FF00D839FF00D749FAF
:1013E000F00D659FF00D9927729FB00DE11DF91F5B
:1013F000639FB00DE11DF91FBD01CF0111240895B8
:1014000097FB092E05260ED057FD04D014D00AD024
:10141000001C38F450954095309521953F4F4F4F23
:101420005F4F0895F6F790958095709561957F4F81
:101430008F4F9F4F0895A1E21A2EAA1BBB1BFD01DF
:101440000DC0AA1FBB1FEE1FFF1FA217B307E407A3
:10145000F50720F0A21BB30BE40BF50B661F771FFB
:10146000881F991F1A9469F76095709580959095DB
:0C1470009B01AC01BD01CF010895FFCF2E
:10147C000102040801000A006400E80310270100BF
:02148C0000005E
:00000001FF
